:101038002025322E5820002053797374656D20487E
:10104800414C54454400204C6F632E205374657006
:10105800706572206572726F7200205379737465BF
:101068006D205245534554002020202E2E2E20500E
:101078006C65617365207761697400204D656368EC
:10108800616E6963616C204572726F720020202066
:101098002E2E2E2053796E6368726F6E697A65649E
:1010A80000202E2E2E205361766500202E2E2E2015
:1010B80045646974002042617365202025332E64DD
:1010C800202D203078255820200020456E61626C44
:1010D800656420002044697361626C656400202E99
:1010E8002E2E20526573657400202E2E2E205379E3
:1010F8007374656D20726573746172747300204334
:101108006F6E6669726D202E2E2E2E2E002053745F
:10111800657070657220417474656E74696F6E00D5
:10112800205A6F6F6D20737769746368202E2E2E96
:101138000020506F7320583A2025342E6400205424
:1011480065737420706173736564202E2E2E0020E1
:1011580054657374206661696C6564202E2E2E00B8
:1011680020466F63757320737769746368202E2E29
:101178002E0020506F7320593A2025342E640053D6
:101188006F6674205265736574202E2E2E00202EF3
:101198002E2E20506C65617365205761697400209C
:1011A8002E2E2E2053656C65637400202E2E2E2063
:1011B80045646974202000202E2E2E2043616E6322
:1011C800656C20496E707574005A4F4D4D2044521D
:1011D800495645520076657273696F6E20312E3418
:1011E80030005045474153555320323030310020AC
:1011F80053447850205820434F4D4D206572726FEC
:1012080072002053447850205920434F4D4D20659B
:1012180072726F72002573205A3A25332E6420208B
:10122800463A25332E642000446D782025332E64F9
:10123800202D2025322E642025322E6420200025E2
:101248007300496E6974205A4F4F4D202E2E2E2060
:1012580000496E697420464F435553202E2E2E00A8
:10126800204D616E75616C20636F6E74726F6C20B7
:10127800000000002052656D6F746520636F6E7406
:10128800726F6C20000000004F7065726174696FA6
:101298006E206D6F6465200000000000444D5820EA
:1012A80061646472657373202020200000000000D0
:1012B80041636F75737469632062656570202000EF
:1012C8000000000052656C6F61642064656661759A
:1012D8006C74730000000000446961676E6F73747A
:1012E8006963732020202000000000004D616E75A6
:1012F800616C0052656D6F74650020204E6F20721E
:101308006563657074696F6E004E6F2044494D4D7A
:101318004552206461746100202020446D78206467
:07132800617461204F4B00CE
:0C27B600044800401454C10CC10EC10DB9
:10000300E4FDEF4E6018EF1F70011E7C66EC600884
:0E0013001CEDF5F0A4FD80F5D2AED2BE80E467
:0100210022BC
:0C278F00EF60091F7E15EE60F71E80FA57
:01279B00221B
:0227EE000022C7
:1025C400AD07AC06300625D2ECC2EEED25E0FDECFD
:1025D40033FCED4C6012ED1D70011C7F0512278F3A
:0D25E400B2EBD2AED2BE80EAC2ECC2EB2256
:1020C400AB07AA06ED14601D1460251460262403D2
:1020D400702D7D64EBAE027802CEC313CE13D8F913
:1020E400FBAA06802B7D32EAC313FAEB13FB802094
:1020F4007D19801C7D0AEB25E0FBEA33FA80117D13
:1021040005EBAE027802C333CE33CED8F9FBAA0670
:10211400D2ECC2EEEB4A6012EB1B70011AAF05124F
:0F212400278FB2EBD2AED2BE80EAC2ECC2EB2262
:0C27C300D2ED0000C2ED7F0112278F2232
:102646007FFFAEE843E80FC2EFC2ECD2EED2ED0058
:1026560030EB0AEF60071FD2AED2BE80F3C2ED00A8
:082666008EE8EF6002D322C3ED
:01266E002249
:10002600AD07C2EC122646D2ED53E8F0EDC4540FEC
:10003600540F42E81227C3D2ED53E8F0ED540F42B5
:05004600E81227C322AF
:0D279C00C2EEC2EFC2EC43078012002622FD
:101C5500C2EEC2EFC2EDC2EC3002097F147E001263
:101C6500000380077F017E00120003D2ED53E8F0E8
:101C750043E8031227C37F057E00120003D2ED530C
:101C8500E8F043E8031227C37F017E00120003D268
:101C9500ED53E8F043E8031227C37F017E001200ED
:101CA50003D2ED53E8F043E8021227C37F017E001B
:101CB5001200037F281200267F0C1200267F0612D1
:101CC50000267F011200267F021200267F027E0079
:041CD50012000322D4
:10273F007F011200267F027E001200037F0212002B
:07274F0026E4FF12279C2283
:0A27DA00D2EFC2EE120026C2EF2279
:102506008B348A358936D2EFC2EEAB34AA35A9367A
:10251600120643FF601712002674012536F536E4CD
:102526003535F5357F017E0012000380DDC2EF22CE
:04253600AC07AB053E
:10253A0074472CF8E6FF12279CE4FAC3EB6480F890
:10254A00EA648098500C7F201227DAD2AED2BE0AF3
:0B255A0080E974472CF8E6FF12279C74
:012565002253
:10277E00300204C2968002D2967F017E00120003C0
:01278E002228
:0527E400D2F8D2F92239
:061CD9008B388A39893ABC
:101CDF00C2F81227EEC2F9EF25E054FEFFE4FEEF43
:101CEF0025E0FF92F8D2F9C2F90EBE08F2D2F8D26F
:101CFF00F9A2F8B39208C2F9200702D208300841BE
:101D0F00E53B603DAB38AA39A93A120643FFE4FE22
:101D1F00EF25E0FF92F8D2F9C2F90EBE08F2D2F821
:101D2F00D2F9A2F8B39208C2F97401253AF53AE450
:101D3F003539F539153B200702D208D2AED2BE8015
:0C1D4F00BCC2F8D2F91227EED2F8A208AC
:011D5B002265
:061B47008B378A38893952
:101B4D00E4FE7D80C2F81227EEC2F9EF25E04401D4
:101B5D00FFE4FCEF25E0FF92F8D2F9C2F90CBC08C6
:101B6D00F2D2F8D2F9A2F8B39206C2F9300648E5DE
:101B7D003A6044E4FFFCD2F930F803ED4207C2F9B4
:101B8D00EDC313FD0CBC08EEAB37AA38A939EF1223
:101B9D000689153AE53A6004C2F88002D2F8D2F906
:101BAD001227EEC2F974012539F539E43538F538C7
:101BBD000ED2AED2BE80B5C2F8D2F91227EED2F84F
:021BCD00AF0661
:011BCF0022F3
:1024D500C20675360A7860A60708A60520061FE518
:1024E50036601B7F017E001200037B007A00796055
:1024F500753B02D2077F50121CD9920680DEA206D8
:0125050022B3
:10249C00C20575280A7860A607ECFF3395E0EF08B3
:1024AC00F6ED08F620051FE528601B7F017E001263
:1024BC0000037B007A007960753B03D2077F5012D2
:0824CC001CD9920580DEA20577
:0124D40022E5
:1026BC007860A6077B007A007960753B01D2077FB2
:1026CC0050121CD97B007A007960753A017F501248
:0526DC001B47E6FF2290
:0222C6008F1B6C
:1022C8007860A61B7B007A007960753B01D2077F96
:1022D80050121CD97B007A007960753A017F501240
:1022E8001B47E6F51CE51B04F67B007A0079607550
:1022F8003B01D2077F50121CD97B007A00796075A8
:102308003A017F50121B47E51CFEE67C002400FFC3
:03231800EC3EFE9A
:01231B00229F
:10231C007B7820940BA20592067F0A7E001225C4BE
:10232C0043E80FD2EED2ECE5E8540FFA30041B2050
:10233C009418EB600A7F0A7E001200031B80F0D217
:10234C00067F0A7E001225C480E5C2EEC2ECC2C133
:06235C00C20CD2B9AF0271
:012362002258
:1026E1007B78209418EB600A7F0A7E001200031B9E
:1026F10080F0D2067F0A7E001225C480E5C2C1C2E5
:032701000CD2B93E
:0127040022B2
:0D27A9003094097F017E0012000380F422AD
:0223A6008F3472
:1023A8007F301226BC8F35E5352431FFAD34122439
:1023B800D50535E535C3940550028001C34003E4D3
:1023C800F535AD357F301224D5E4FBD2067F1E7E6D
:0F23D800001225C47FC87E001200030BBB06EC69
:0123E70022D3
:102208007F301226BC8F101510E4F511E510C39429
:102218000550028001C34003751004E5102431FF06
:102228001226BC74122511F8A60715100511E51120
:10223800C3940540D7E4F511E51175F003A42460B3
:10224800F9E4FAFB752FFF753010753138741225D3
:1022580011F8E6753200F5331208040511E511C3CB
:04226800940540D4C5
:01226C00224F
:10270500E4FD7F301224D5E4F51FE51F2431FF7D5C
:0D271500FF1224D5051FE51FC3940540EDFC
:012722002294
:1025F10012273F7F4012279C7B007A0079601225C9
:10260100067F1412279C7BFF7A10793F1225067FE3
:0B261100F21223A6D2AED2BE80FA2245
:10272300ED14FEEED39400400EEF2E14F8E6FDEF09
:0B2733002EF8A6051E80ECA807A603E8
:01273E002278
:10269600E4F51DF51EFEEEC39D5010A807E6251EA7
:1026A600F51EE4351DF51D0E0F80EBED7C00AE1D0D
:0526B600AF1E12070237
:0126BB0022FC
:10246200ED14FEC3EE64809480402E7D01D3EE64B1
:1024720080F8ED648098501EEF2DF8E6FCE814F821
:10248200E6FBD39C400DA903EF2D14F8A604EF2D13
:09249200F8A6010D80D71E80CAD6
:01249B00221E
:02259600A90793
:10259800ED14FFEFD394004019EF25E02924FEF84D
:1025A800E6FC08E6FDEF25E029F8A60408A6051FC5
:0B25B80080E1AF01A807A60208A603FF
:0125C30022F5
:10261C00E4F529F52AFEEEC39D5014A807E6FA0846
:10262C00E6252AF52AEA3529F5290E0F0F80E7ED64
:09263C007C00AE29AF2A1206ADA4
:012645002272
:02275600A905D3
:10275800E4FEEEC399500CA807A60208A6030E0FC4
:032768000F80EFF0
:01276B00224B
:1025660012273F7F4012279C7BFF7A10794E122557
:10257600067F1412279C7BFF7A1079621225067F4C
:10258600F11223A6D2067FD07E071225C480FE2232
:041BD0008F298D2AA2
:101BD400752B05752C05C20378607680087681081C
:101BE40076827960E7182624827863F6200343E539
:101BF4002C603FE529C313452AFF7B007A007960F6
:101C0400753B04D207121CD94011E52B600DD20696
:101C14007F0A7E001225C4152B80D87F0412278FDB
:101C240020F904D20380077F327E00120003152CB2
:101C340080BA7FC87E00120003E52B6006E52C60A5
:101C440002D322D2067FD07E071225C4122566C392
:011C5400226D
:081914008F2C8D2D8A2E8B2FE4
:10191C00753005753105C20378607690E52EFF337E
:10192C0095E0EF08F6AF2FE52F08F6FF7960E71882
:10193C00262F7863F6200343E531603FE52CC31373
:10194C00452DFF7B007A007960753B04D207121C91
:10195C00D94011E530600DD2067F0A7E001225C4F5
:10196C00153080D87F0412278F20F904D20380070A
:10197C007F327E00120003153180BA7FC87E0012C0
:10198C000003E5306009E5316005AE2EAF2F221261
:06199C0025667EFF7FFFBF
:0119A2002222
:041ED8008F2C8D2D91
:101EDC00753005753105C203786076A008A6030835
:101EEC00A62F7960E71826252F7863F6200343E5A3
:101EFC0031603FE52CC313452DFF7B007A007960E0
:101F0C00753B04D207121CD94011E530600DD20686
:101F1C007F0A7E001225C4153080D87F0412278FCB
:101F2C0020F904D20380077F327E001200031531A2
:101F3C0080BA7F647E00120003E5306006E53160F4
:071F4C0002D322122566C337
:011F5300226B
:041881008F288D29F6
:10188500752E05752F05C202786076C0AE02AF03CE
:101895007C007D641207027861A607AE2CAF2D7C13
:1018A500007D641207027862EFF67960E718262F4B
:1018B5007863F6200243E52F603FE528C3134529E9
:1018C500FF7B007A007960753B04D207121CD94072
:1018D50011E52E600DD2067F0A7E001225C4152E55
:1018E50080D87F0412278F20F904D20280077F3227
:1018F5007E00120003152F80BA7F647E001200035C
:0E190500E52E6006E52F6002D322122566C390
:0119130022B1
:041D5C008F288D2916
:101D6000752D05752E05C202786076B008A603E5CC
:101D70002BC313E52C13FF08F67960E718262F789C
:101D800063F6200243E52E603FE528C3134529FF93
:101D90007B007A007960753B04D207121CD9401190
:101DA000E52D600DD2067F0A7E001225C4152D8018
:101DB000D87F0412278F20F904D20280077F327E59
:101DC00000120003152E80BA7F647E00120003E526
:0D1DD0002D6006E52E6002D322122566C3A9
:011DDD0022E3
:041F54008F288D291C
:101F5800752C05752D05C202786076D008A6030891
:101F6800A62B7960E71826252B7863F6200243E52F
:101F78002D603FE528C3134529FF7B007A0079606F
:101F8800753B04D207121CD94011E52C600DD2060E
:101F98007F0A7E001225C4152C80D87F0412278F53
:101FA80020F904D20280077F327E00120003152D2B
:101FB80080BA7F647E00120003E52C6006E52D6080
:071FC80002D322122566C3BB
:011FCF0022EF
:041DDE008F178D18B6
:101DE200751905751A05C20F786076E0EA08F6AF34
:101DF20003EB08F67960E718262F7863F6200F4385
:101E0200E51A603FE517C3134518FF7B007A007996
:101E120060753B04D207121CD94011E519600DD23E
:101E2200067F0A7E001225C4151980D87F04122766
:101E32008F20F904D20F80077F327E001200031533
:101E42001A80BA7F647E00120003E5196006E51A63
:081E52006002D322122566C3D1
:011E5A002265
:041E5B008F2C8D2D0E
:101E5F00752E05752F05C20478607620300304E6D1
:101E6F004401F6786176AA0876BB7960E7182624D4
:101E7F00BB7863F6200443E52F603FE52CC3134581
:101E8F002DFF7B007A007960753B04D207121CD9B5
:101E9F004011E52E600DD2067F0A7E001225C41573
:101EAF002E80D87F0412278F20F904D20480077F59
:101EBF00327E00120003152F80BAE52E6006E52F43
:081ECF006002D322122566C354
:011ED70022E8
:0819A3008F2C8D2D8A2E8B2F55
:1019AB00753205753305C203D3E52F9531E52E95B9
:1019BB0030400685302E85312F78607638E52E083D
:1019CB00F6AF2FE52F08F6FF7960E718262F78631F
:1019DB00F6200343E533603FE52CC313452DFF7B16
:1019EB00007A007960753B04D207121CD94011E5CF
:1019FB0032600DD2067F0A7E001225C4153280D8C4
:101A0B007F0412278F20F904D20380077F327E00D8
:101A1B00120003153380BAE5336005AE2EAF2F22CB
:031A2B001225661B
:011A2E002295
:0416CF008F298D2AA8
:1016D300753105753205C205E52E2BE52D3AC39408
:1016E300005009C3E49BF52EE49AF52DE52E2BFF5C
:1016F300E52D3AFED3EF9530EE952F400AE5309B6A
:10170300F52EE52F9AF52DD3E52E9400E52D648073
:101713009480400878607611D20480067860761051
:10172300C2043003067860E64404F6AF2EAE2D12F1
:10173300276C8E2D8F2EE52E452D70030217C3E5E2
:101743002DFF3395E0EF7861F6AF2EE52E08F6FF17
:101753007960E718262F7863F6200543E532603F6A
:10176300E529C313452AFF7B007A007960753B04A2
:10177300D207121CD94011E531600DD2067F0A7ED3
:10178300001225C4153180D87F0412278F20F90455
:10179300D20580077F327E00120003153280BAE53E
:1017A3003260197F037E00120003300405AE2DAFB3
:1017B3002E22C3E4952EFFE4952DFE2212256622E8
:0417C3007E007F0025
:0117C70022FF
:101FD000300418AD4FAC4E7F1012249CAD4D7F23C2
:101FE0001224D5AD4C7F211224D5227F101226BC9D
:101FF000EF7F00FEC006C0077F111226BCEFFDD0A8
:10200000E02DF54FD0E03400F54EC3E54F9401E5E7
:102010004E9400400BD3E54F94FFE54E94014006EB
:10202000754E00754F017F231226BC8F4DD3E54DB1
:10203000648094815009C3E54D648094805003E42A
:0A204000F54D7F211226BC8F4C22C3
:0B27CF0075988075A910C298C299226D
:102427008F27752FB4E4FBAD277FB0121ED8752B0D
:1024370001752C187B20AD277FB0121D5C752C030E
:10244700752DE87B907A01AD277FB0121881752B27
:0B245700807B78AD277FB0121F54225D
:0214B4008F297E
:1014B600752A4E752B20EF75F00FA4244AF9741285
:1014C60035F0FA7BFF1225067F4012279C7BFF7AB8
:1014D600107970122506E52914604104707A30B23D
:1014E600777B347A08E4FD7FB0121914C203E4FD59
:1014F6007FB0121E5B30B217E52B452A60117F01C3
:101506007E00120003E52B152B7002152A80E6C219
:10151600F87F017E00120003D2F8803C30B3397B9D
:10152600347A087D017FB0121914C2037D017FB0A1
:10153600121E5B30B317E52B452A60117F017E0032
:10154600120003E52B152B7002152A80E6C2F87FE0
:10155600017E00120003D2F8E52B452A701A7F108F
:101566001223A6752FFF7530107531837B007A0024
:1015760079601208041225F17F1412279C7BFF7AEA
:101586001079951225067F647E00120003753008D7
:101596007531347B287A00AD297FB01219A37F20DC
:1015A6007E03120003752FFFE4FBAD297FB0121EE8
:1015B600D812273FE4FBFAAD297FB01219147E003A
:0215C6007F00A4
:0115C8002200
:03004B000227E9A0
:0527E900D20CC2B93260
:0300230002219E19
:10219E00C0E0C0D075D008309A41300E56300D18C0
:1021AE00C20DE59960057556018048755602E551D8
:1021BE00155170021550803BE5514550600AE551AE
:1021CE00155170021550802B74582557F8A699E5B5
:1021DE005760041557801CC20E8018E599700F8544
:1021EE004E50854F51755701D20DD20E8005C20E3D
:0A21FE0075560AC298D0D0D0E03226
:101A2F00C203D204A203920512231CEF6402607B4F
:101A3F00BF040E154DC3E54D648094805003E4F54B
:101A4F004DBF080E054DD3E54D648094814003755D
:101A5F004D01EF640170287F5412279C7BFF7A1091
:101A6F0079A9122506D204121FD07FE87E03120037
:101A7F00037F5412279C7BFF7A1079B31225067FC0
:101A8F004012279CAF4DEF3395E0FE7C007D141282
:101A9F00069B74682FF974123EFA7BFF122506E538
:0B1AAF004C24FF92031227A9021A31F9
:011ABA002209
:1017C800C204C20512231CEF64027003021873BF1F
:1017D8000417054FE54F7002054ED394FFE54E946C
:1017E800014006754E00754F01BF0819E54F154FAA
:1017F8007002154EC3E54F9401E54E9400500675EE
:101808004E01754FFFEF640170287F5412279C7BAF
:10181800FF7A1079A9122506D204121FD07FE87E1C
:10182800031200037F5412279C7BFF7A1079B312AE
:1018380025067F4012279C752FFF7530107531BD26
:10184800854E32854F33854E34854F357B007A007F
:1018580079601208047B007A0079601225067FC837
:101868007E001200031227A90217C8E54C24FF9234
:08187800067F0A7E001225C460
:011880002245
:10204A00C203D204A203920512231CEF6402606940
:10205A00EF64046003BF080CE54C70047E01800243
:10206A007E008E4CEF640170287F5412279C7BFF00
:10207A007A1079A9122506D204121FD07FE87E03AE
:10208A001200037F5412279C7BFF7A1079B3122522
:10209A00067F4012279CE54C600B7BFF7A1079D2B1
:1020AA0012250680097BFF7A1079DC122506E54C99
:0920BA0024FF92031227A980897A
:0120C30022FA
:10213300C203D204A203920512231CEF6402605A65
:10214300EF6401703C754D01F54E754F01754C01FF
:102153007F5412279C7BFF7A1079E6122506D2045E
:10216300121FD07FE87E031200037F5412279C7B4B
:10217300FF7A1079F11225067FE87E0312000380AF
:10218300FE7F4012279C7BFF7A117906122506E514
:0A2193004C24FF92031227A9809844
:01219D00221F
:10132F0012273F7F4012279C7BFF7A1179151225D8
:10133F0006E4FD7FB0121BD07D017FB0121BD012CF
:10134F00273FE4FF1214B48E528F537F011214B44F
:10135F008E548F5512273F7F4012279C7BFF7A11A7
:10136F007928122506E4F5287F5412279C752FFF44
:10137F007530117531398552328553337B007A00C0
:10138F0079601208047B007A007960122506752DAA
:10139F0001752E90752F08753034C203AB53AA52C6
:1013AF00E4FD7FB01216CFEF2553F553EE3552F50E
:1013BF00527F0A7E0012000320FF06D2AED2BE80FB
:1013CF00F77FC87E001200030528E528C394054067
:1013DF00977F5412279CE553B4D010E552B4070BF6
:1013EF007BFF7A11794612250680097BFF7A1179E6
:1013FF00571225067FD07E0712000312273F7F402A
:10140F0012279C7BFF7A117968122506E4F5287F55
:10141F005412279C752FFF75301175317A85543210
:10142F008555337B007A0079601208047B007A00BF
:10143F007960122506752D01752E2C752F057530C7
:10144F00F0C203AB55AA547D017FB01216CFEF2522
:10145F0055F555EE3554F5547F0A7E0012000320E2
:10146F00FF06D2AED2BE80F77FC87E001200030502
:10147F0028E528C3940540977F5412279CE555B45F
:10148F00DC10E554B4050B7BFF7A11794612250663
:10149F0080097BFF7A1179571225067FD07E0712BC
:0414AF00000380FEB8
:0114B3002216
:1023E80012273FE4FF12279C7BFF7A117987122579
:1023F800067F4012279C7BFF7A11799612250612D8
:1024080026E1E4FBE54C24FF92067F1E7E001225A0
:0E241800C47FC87E001200030BBB06E880FEE6
:012426002293
:1015C900E4F527C20212273FE4FF12279CAF27EF59
:1015D9003395E0FE7C007D1412069B74902FF974FC
:1015E900123EFA7BFF1225067F5412279C7BFF7A55
:1015F9001179A71225061226E11227A9D204E54C72
:1016090024FF920512231CEF640270030216C7BF60
:10161900040E1527C3E527648094805003E4F52759
:10162900BF080A0527E527B40503752704EF6401F8
:1016390070667F5412279C7BFF7A1179B3122506B5
:10164900E527146012146014146016146018240439
:101659007019121A2F80291217C8802412204A8063
:101669001F122133801A12132F80157F4012279CD5
:101679007BFF7A1179BF1225067FE87E03120003EA
:101689007D147F021225367F5412279C7BFF7A1125
:1016990079A71225061226E1E4FF12279CAF27EF4E
:1016A9003395E0FE7C007D1412069B74902FF9742B
:1016B900123EFA7BFF1225061227A90216057D1490
:0516C9007F041225362C
:0116CE0022F9
:10226D0020022B7F797D0312261C8E278F28EF6588
:10227D00537003EE65526040753008753134AB28EC
:10228D00AA27E4FD7FB01219A38E528F53227F7FB0
:10229D007D0312261C8E278F28EF65557003EE6582
:1022AD005460157530057531F0AB28AA277D017F77
:0822BD00B01219A38E548F55D5
:0122C50022F6
:10236300200224E528AE277803C333CE33CED8F931
:10237300FDAC06E528AE277802CEA2E713CE13D82C
:10238300F82DFFEE3CFE22E52825E0FDE52733FC92
:10239300E528AE277802C333CE33CED8F92DFFEE2E
:0323A3003CFE22DB
:100C17007523FA75241E7525FFE47887F6C200F55B
:100C270087F5D01227E41227CFD2BED297F556C246
:100C370004121FD07E007F007D027B007A00795866
:100C470012077CD2B9C2CDD2AFD29CC298D2ACD255
:100C570002121C55E4FF12279C7BFF7A1179D112EF
:100C670025067F4712279C7BFF7A1179DD1225061F
:100C77007F5C12279C7BFF7A1179EA122506D20244
:100C870012277E7FB87E0B12000312273F7E007F5C
:100C9700067D007B007A00795A12077CE4FD7FB05D
:100CA700121BD04015752FFF7530117531F77B007A
:100CB7007A0079601208041225F17D017FB0121BBA
:100CC700D04015752FFF75301275310A7B007A00F9
:100CD70079601208041225F1D2067FC87E0012251A
:100CE700C4E4FF122427E4FF1214B48E528F537FFB
:100CF700011224277F011214B48E548F55E5256005
:100D0700041525800B7525FFE4F524C202121C5536
:100D1700E4FF12279CAF4DEF3395E0FE7C007D0783
:100D270012069B74F42FF974123EFA7BFFC003C0BE
:100D370002AE52AF537D151206ADAA06AB07AE54ED
:100D4700AF557C007D0F1206AD8E378F388A358BF5
:100D570036D002D0038B328A338934752FFF753032
:100D67001275311D7B007A0079601208047B007AC6
:100D7700007960122506300C23D20212277E7523D4
:100D8700FAC204E54C24FF920512231C8F22BF03ED
:100D9700031223E8E522B401031215C9E4F526E599
:100DA7002675F003A4245AFFC3740195262458F826
:100DB700E6FB7D03122723E52675F003A4245AF9E1
:100DC700E4FAFB78607C00FDFE7F0312061D7F605E
:100DD7007D031224627861E6FF74852526F8A6074D
:100DE7000526E526C3940240B67F4112279C752F3E
:100DF700FF753012753130854E32854F33AC59E46B
:100E07001200F87B337A33792378401200511201AC
:100E17002C8E348F35AC58E41200F87B337A337953
:100E270023784012005112012C8E368F377B007ABF
:100E37000079601208047B007A007960122506D2D7
:100E470001E52460041524803A7F5A12279CE55651
:100E570075F00FA42402F9741335F07532FFF533DA
:100E67008934752FFF7530127531477B007A007909
:100E7700601208047B007A00796012250675241E2B
:100E8700E4F556E54D147003020FCC04600302101D
:100E970014C204C20512231C8F22D2007887E6C32E
:100EA700940C500106E52224FA7003020F4824FE31
:100EB700603924FE7003020F6724FE606F24FE7002
:100EC70003020FA7240A6003020FBD7887E67E009E
:100ED7002553FBEE3552FA753008753134E4FD7F42
:100EE700B01219A38E528F53020FC37887E6FF7E85
:100EF70000D3E5539FE5529E401CE5539FFBE55207
:100F07009EFA753008753134E4FD7FB01219A38E4F
:100F1700528F53020FC3753008753134E4FBFAFD65
:100F27007FB01219A38E528F53020FC37530087505
:100F37003134E4FBFAFD7FB01219A38E528F538030
:100F47007B7887E67E002555FBEE3554FA7530052C
:100F57007531F07D017FB01219A38E548F55805CD7
:100F67007887E6FF7E00D3E5559FE5549E401BE555
:100F7700559FFBE5549EFA7530057531F07D017F6D
:100F8700B01219A38E548F5580327530057531F024
:100F9700E4FBFA7D017FB01219A38E548F55801C94
:100FA7007530057531F0E4FBFA7D017FB01219A3A6
:100FB7008E548F558006E47887F6C2007F197E002D
:100FC7001200038048C2027885E6752700F52812CB
:100FD7002363AA06AB077F797D03122596C2021207
:100FE700226D7F147E00120003D2027886E67527F1
:100FF70000F528122363AA06AB077F7F7D0312251E
:1010070096D20212226D7F507E0012000330000438
:10101700C2008017E523600415238005C20212274A
:101027007EE54D70067F46FE120003C297020D044F
:011037002296
:10004E000201A2EC5D046005E859047003020198F8
:10005E00120163580460F6EC4860F2EC7004FDFE89
:10006E00FF22C860DB2481C85009C3986002500685
:10007E0002019F9850CAF582E9294B4A7005AB825E
:10008E0002018E75F0007C1A7880C3EF9BEE9AED1C
:10009E0099400DC3EF9BFFEE9AFEED99FDE842F0FD
:1000AE00DC23ACF0D0E0FFD0E0FED0E0FDAB822050
:1000BE00E7101BEB60BAEC2CFCEF33FFEE33FEEDDA
:1000CE0033FD02017AE803F830E705C0F075F00061
:1000DE00EF2FFFEE33FEED33FD40B830E7C280AABE
:1000EE0075F020800E75F010800575F0087D007E8D
:1000FE00007F003392D530D503120738EC33401011
:10010E00EF33FFEE33FEED33FDEC33FCD5F0ED2295
:0E011E00E5F0247EA2D513CC92E7CDCEFF22D1
:10012C00EDD2E7CD33EC3392D524814006E4FFFECB
:10013C00FDFC22FCE4CFCECDCC24E0501174FF802A
:10014C00EDC3CC13CCCD13CDCE13CECF13CF0470C7
:07015C00F030D5DE02073888
:1007A800E543242FF8E6054322782C300A02782FF7
:1007B800E475F0011207460206432003EB7F2ED2B0
:1007C800038018EF540F2490D43440D4FF30070B23
:1007D800EF24BFB41A0050032461FFE544600215FA
:1007E800440547E54770020546300A0D782CE47544
:1007F800F001120746EF02068902266F7403D20A37
:100808008003E4C20AF5438B2C8A2D892EE4F54433
:10081800F546F547E54460077F201207E380F57544
:1008280045FFC204C203C205C206C208C209C20B00
:100838001207B1FF700D300A057F001207F4AF47A9
:10084800AE4622B4255FC2D5C2071207B1FF24D035
:10085800B40A00501A75F00A784430D50508B6FF76
:100868000106C6A426F620D5047002D20680D92433
:10087800CFB41A00EF5004C2E5D207020AE1D2044D
:1008880080C6D20380C0D20580BCD2D580BAD20837
:1008980080B47F201207E32005077401B5440040A7
:1008A800F11207A8FF1207E302081CD20BD2098035
:1008B800951207A8FB1207A8FA1207A8F94A4B7065
:1008C8000679D87A0B7BFF20052EE544602A7E0046
:1008D8008E8275830012065C60060EEE654570F028
:1008E800C2D5EBC0E0EAC0E0E9C0E0EE120B41D0AF
:1008F800E0F9D0E0FAD0E0FB120643FF60AAEBC0B3
:10090800E0EAC0E0E9C0E01207E3D0E02401F9D052
:10091800E03400FAD0E0FBE5450460DCD545D98039
:1009280087D20580A2120B2460F7E54570010412F6
:1009380001ADA945600DE545600914F545120BCBDD
:10094800EF60F3EA30E702F404C3995077EAF4253C
:10095800450430E701E404F545800D120B2460C11D
:10096800EA054525451201ADEA7842F630E701E48B
:10097800254504D5450420080114120B41E4C0E0C4
:10098800120BCB7842E6601320E70714F61207CB68
:10099800802204F6D0E014C0E07F001207CBE545C2
:1009A80060071207C21545800B3008031207C2D032
:1009B800E002081CD0E00480C5120B2460A0E545C5
:1009C800041201AD7842EAF6E54520080260010408
:1009D8002404120B4174FF04C0E0120BCB1207CBA6
:1009E800E54520080260031207C2D0E0B545E87F5C
:1009F800451207D57842E67F2B30E7047F2DF404B3
:100A0800C0E01207E3D0E075F00A84C0F01207CC0A
:100A1800D0E01207CC02081C791080027908C209BC
:100A2800C20B8008D2D5790A8004790AC2D5E54577
:050A3800047002F54509
:100A3D00E4FAFDFEFF1207A8FC7B08200413120741
:100A4D00A8FD7B1030030A1207A8FE1207A8FF7B32
:100A5D0020EC3382D592D55013C3E43003069FFFAB
:100A6D00E49EFEE42004039DFDE49CFCE4CBF8C26F
:100A7D0004EC700CCFCECDCCE824F8F870F38017D1
:100A8D00C3EF33FFEE33FEED33FDEC33FCEB33FB05
:100A9D00994002FB0FD8E9EB300405F8D0E0C448CB
:100AAD00B204C0E00AEC4D4E4F78207B0070C2EAD4
:100ABD00B5450040BCC0E0120B43D0F0D0E020049F
:100ACD0004C4C0E0C4B204C0F01207CCD0F0D5F01D
:100ADD00EB02081C12075608B9530A2058088A4C15
:100AED000886420A244F0A2C440A2C49089F430ABF
:100AFD00325509634609C145092D470BF850088E3B
:100B0D002D08922E08B52B08962308B3200BE62A44
:100B1D00084E48000008ADE545B4FF0375450612C3
:100B2D0007A8FC1207A8FD1207A8FE1207A8FF7858
:100B3D003B0201DC790AA2D5200614300809B91050
:100B4D00020404B9080104A2D520090250010420B1
:100B5D0005689205B544005034C0E07F2030061979
:100B6D007F30A20572097208500F120B9AC205C28E
:100B7D0009C208C20B7F30800F300803E9C0E012B4
:100B8D0007E3300803D0E0F9D0E0B544CC300817C6
:100B9D007F30B9100C1207E37F583007077F78803C
:100BAD0003B908031207E33005057F2D0207E37F24
:100BBD0020200BF87F2B2009F322920580CF7F0098
:100BCD00B407005005243BF8E6FF22286E756C6CC7
:100BDD0029002D50434958D2041207A83004F8C2F9
:100BED0004784430D50108F602084E1207A82403F4
:100BFD00B405004001E4900BDF931207D4743A1250
:0A0C0D0007D4D206754404020A2041
:10016300E9D2E7C933E833F892D5EDD2E7CD33ECE2
:0701730033FC5002B2D5225B
:10017A00EC30E7100FBF000C0EBE00080DBD0004E6
:10018A000BEB6014A2D5EB13FCED92E7FD2274FF92
:10019A00FCFDFEFF22E480F8A2D574FF13FC7D80EB
:0301AA00E480EFFF
:1001AD00F920E72824F950037907E4F42402FB1819
:1001BD00DBFDE624FB5014E9600DE4F618E604F6C9
:0F01CD00B40A08E4F6D9F57401F60A22C2D52265
:1001DC00ED33EC3392D5FA602AB4FF33EDC2E77BF2
:1001EC00FF60067A027901E4227A02790A20D504AA
:1001FC007A027905224E614E002B494E46002D495C
:10020C004E4600E47A08F608DAFC7B00740722E814
:10021C00C0E0ECC0E0EDC0E0EEC0E0EFC0E0EA759D
:10022C00F010A4CAABF075F04DA42BFBE435F0FC38
:10023C00EA2410FAEB34C5FBEC34D9FCEDC2E7FF31
:10024C0075F056A4F42411C5F0F434C58FF0A42A2B
:10025C00E5F03BE43CF620E71412050DD0E0FFD0AE
:10026C00E0FED0E0FDD0E0FC1200518014F404124A
:10027C00050DD0E0FFD0E0FED0E0FDD0E0FC120395
:10028C00D7D0E0F8E6FAEDD2E7CD33EC332482FB9D
:10029C00E4C3CF33CFCE33CECD33CD33DBF37B07BB
:1002AC0075F00A846004F6081B0AE5F0F6088FF076
:1002BC00740AA4FFACF08EF0740AA42CFEACF050BF
:1002CC00010C8DF0740AA42CFDE435F0F608DBDE8D
:0302DC0074072282
:1002DF00020198E86480F8E933E83360110460F0B4
:1002EF00ED33EC337009E8FCE9FDEAFEEBFF220485
:1002FF0060DED3EB9FEA9EE99DE8C2E78CF0C2F780
:10030F0095F0400CE8CCF8E9CDF9EACEFAEBCFFB4B
:10031F0012016385D0F05804700320D5B3E8047040
:10032F00075002B2D50201A292D5EC0460F7E4CCDB
:10033F00C0E0C398F8603B94186008400DD0E0FB14
:10034F0002017AE4FBFAC9FC8028E830E406E4C92C
:10035F00FBE4CAFCE830E305E4C9CACBFCE8540768
:10036F006010F8C3E913F9EA13FAEB13FBEC13FC73
:10037F00D8F130F52FC3E49CFCEF9BFFEE9AFEED16
:10038F0099FDD0E0FBEF4E4D4C701222DB030201C2
:10039F009FEC2CFCEF33FFEE33FEED33FDED30E73A
:1003AF00EB02017AEF2BFFEE3AFEED39FDD0E0FBC9
:1003BF0050130BBB00030201A2ED13FDEE13FEEF72
:0803CF0013FFEC13FC02017A9C
:1003D700EC4D6011E8497017ED33EC3304600DE420
:1003E700FCFFFEFD22E933E8330470F8020198129E
:1003F700016358046009E4CC24815006285009029F
:1004070001A228400302019FC0E0EB4A7044B98073
:1004170006D0E0FB02018EEF4E701CBD8008EBFF9B
:10042700EAFEE9FD80EBE98DF0A4FEE5F00204C0E9
:10043700E9CDF9EAFEEBFFEF89F0A4FCE5F0CE8900
:10044700F0A42EFFE435F0CD89F0A42DFEE435F0BD
:100457008067EF4E7005BD80D780C3EF8BF0A4ACEB
:10046700F0EE8BF0A42CFCE435F0F8EF8AF0A42C26
:10047700E5F038FCE433CB8DF0A42CFCE5F03BF839
:10048700EE8AF0A42CFCE5F038F8E433CF89F0A429
:100497002CFCE5F038CF3400CE89F0A42FFFE5F02F
:1004A7003EFEE433C98DF0A42EFEE5F039CD8AF087
:1004B700A42FFFE5F03EFEE43DFD33D0E0FB5007FF
:1004C7000BBB000F0201A2EC2CFCEF33FFEE33FE57
:0604D700ED33FD02017A85
:1004DD003F8000004120000042C80000447A000027
:1004ED00461C400047C35000497424004B189680A9
:1004FD004CBEBC205A0E1BCA6753C21C749DC5AEA0
:10050D00FB60065407601C232312053BEB54386037
:10051D00091205271205361203D7ECF8EDF9EEFA9C
:10052D00EFCB22EB12053680F1543803241C9004D6
:10053D00DDFE93FC0EEE93FD0EEE930ECE93FF2299
:03000000021ABB26
:0C1ABB00787FE4F6D8FD758187021B02DD
:10054D00E709F608DFFA8046E709F208DFFA803E90
:10055D0088828C83E709F0A3DFFA8032E309F6087D
:10056D00DFFA8078E309F208DFFA807088828C83E5
:10057D00E309F0A3DFFA806489828A83E0A3F60899
:10058D00DFFA805889828A83E0A3F208DFFA804C73
:10059D0080D280FA80C680D4806980F2803380104A
:1005AD0080A680EA809A80A880DA80E280CA8033B3
:1005BD0089828A83ECFAE493A3C8C582C8CCC5832B
:1005CD00CCF0A3C8C582C8CCC583CCDFE9DEE780FB
:1005DD000D89828A83E493A3F608DFF9ECFAA9F07A
:1005ED00EDFB2289828A83ECFAE0A3C8C582C8CCD0
:1005FD00C583CCF0A3C8C582C8CCC583CCDFEADEE9
:10060D00E880DB89828A83E493A3F208DFF980CC4A
:10061D0088F0EF60010E4E60C388F0ED2402B40443
:10062D000050B9F582EB2402B4040050AF232345EA
:06063D00822390059D736D
:10064300BB010689828A83E0225002E722BBFE02B5
:09065300E32289828A83E49322E8
:10065C00BB010CE58229F582E5833AF583E0225053
:10066C0006E92582F8E622BBFE06E92582F8E2229D
:0D067C00E58229F582E5833AF583E49322B7
:10068900BB010689828A83F0225002F722BBFE0150
:02069900F3224A
:10069B00EF8DF0A4A8F0CF8CF0A428CE8DF0A42E73
:0206AB00FE222D
:1006AD00BC000BBE0029EF8DF084FFADF022E4CC31
:1006BD00F875F008EF2FFFEE33FEEC33FCEE9DECFA
:1006CD00984005FCEE9DFE0FD5F0E9E4CEFD22ED40
:1006DD00F8F5F0EE8420D21CFEADF075F008EF2F8A
:1006ED00FFED33FD4007985006D5F0F222C398FD7B
:0506FD000FD5F0EA2218
:10070200C2D5EC30E709B2D5E4C39DFDE49CFCEE12
:1007120030E715B2D5E4C39FFFE49EFE1206ADC3D7
:10072200E49DFDE49CFC80031206AD30D507C3E4D2
:060732009FFFE49EFE2281
:0E073800C3E49FFFE49EFEE49DFDE49CFC22D2
:10074600FAE6FB0808E6F925F0F618E6CA3AF622B4
:10075600D083D082F8E4937012740193700DA3A332
:1007660093F8740193F5828883E473740293686046
:06077600EFA3A3A380DF46
:10266F00EFB40A07740D12267A740A309811A899DC
:10267F00B8130CC2983098FDA899C298B811F630CB
:07268F0099FDC299F59922A3
:10276C00C3EE6480948040028007C3E49FFFE49E24
:02277C00FE223B
:10077C00EF4E6012EF60010EEDBB010B89828A8394
:10078C00F0A3DFFCDEFA2289F05007F709DFFCA9A1
:0C079C00F022BBFEFCF309DFFCA9F022F8
:101AC700020C17E493A3F8E493A34003F68001F212
:101AD70008DFF48029E493A3F85407240CC8C33320
:101AE700C4540F4420C8834004F456800146F6DFEF
:101AF700E4800B01020408102040809027B6E47EA2
:101B0700019360BCA3FF543F30E509541FFEE493E3
:101B1700A360010ECF54C025E060A840B8E493A3AA
:101B2700FAE493A3F8E493A3C8C582C8CAC583CAD5
:101B3700F0A3C8C582C8CAC583CADFE9DEE780BE8D
:0127C2000016
:00000001FF
